:100000007DC00000A2C00000A0C000009EC0000093
:100010009CC000009AC0000098C0000096C000007C
:1000200094C0000092C0000090C000008EC000008C
:100030008CC000008AC0000088C0000086C000009C
:100040000C94120A82C0000084C70000BCC70000E4
:100050007CC000007AC0000078C0000076C00000BC
:1000600074C0000072C00000030405000102040314
:100070000506073F065B4F666D7D077F6F777C58EF
:100080005E79713D74041E703855545C7367506D11
:10009000781C0C6A49725B004049521018080C0425
:1000A000444060202101030200000007000201001B
:1000B0000003040600000000000000000102040824
:1000C00010204080010204081020010204081020C2
:1000D00004040404040404040202020202020303EE
:1000E0000303030300000000250028002B0000008C
:1000F0000000240027002A002F039D0811241FBEA2
:10010000CFEFD8E0DEBFCDBF11E0A0E0B1E0EAEE76
:10011000F8E102C005900D92A835B107D9F722E0A9
:10012000A8E5B1E001C01D92A535B207E1F710E0E6
:10013000CCEFD0E004C02297FE010E94630CC83FC0
:10014000D107C9F788D20C94DA0B5ACFFF920F93DC
:100150001F93CF93DF930CE111E0C5E6D0E0BE0121
:100160008EE991E021D5F82EBE01615071098EE92A
:1001700091E01AD56F2D0E940D0AF8018193919399
:100180008F012296CB37D10551F7DF91CF911F9187
:100190000F91FF900895CF93DF9360E076E98CE7AD
:1001A00091E004D56FE173E08CE791E0D9D5CEDF23
:1001B000CCE1D1E0699179914AE050E082EA91E0A6
:1001C0000E94B20981E0C633D807A1F789E591E022
:1001D00049D28AE591E073D2529A539A549A5A9A24
:1001E000559A5D988AE591E098D48AE591E095D496
:1001F0008AE591E092D48AE591E08FD48AE591E096
:100200008CD48AE591E089D48AE591E086D48AE5A8
:1002100091E0DF91CF9181C4AF92BF92CF92DF92F4
:10022000EF92FF920F931F93CF93DF938AE591E0B4
:1002300074D460E08AE591E05DD2BC01882777FD47
:100240008095982F1F921F921F922BE02F93A12C25
:10025000B12C6501E12C14E0F12E00E010E020E06B
:1002600030E0A9010E94C809C62F669570E08AE5B2
:1002700091E00AD30F900F900F900F90C0FF02C033
:1002800061E001C060E08AE591E006D361E08AE5C3
:1002900091E04DD4882309F45CC089E591E0EED16A
:1002A0008C01FCE1EF2EF1E0FF2EC0E0D0E0F70181
:1002B000419151917F010417150708F444C00417B8
:1002C000150781F4BE01759567958AE591E0DCD24A
:1002D000C0FF02C061E001C060E08AE591E0DCD2CD
:1002E00062E02EC06E018FEFC81AD80A20813181DA
:1002F000241B350B36952795240F351F2017310702
:1003000080F4B601759567958AE591E0BDD2C0FE8F
:1003100002C061E001C060E08AE591E0BDD263E027
:100320000FC0BE01759567958AE591E0ADD2C0FF1B
:1003300002C061E001C060E08AE591E0ADD261E019
:100340008AE591E023D22196CB30D10509F0AFCFD9
:1003500015C060E08AE591E019D260E08AE591E09D
:10036000F0D3882359F0DF91CF911F910F91FF9027
:10037000EF90DF90CF90BF90AF900BC0DF91CF9107
:100380001F910F91FF90EF90DF90CF90BF90AF90B3
:100390000895AF92BF92CF92DF92EF92FF920F93A8
:1003A0001F93CF93DF93C4E0CC2EC1E0DC2E0CE191
:1003B00011E0E12CF12CAA24AA9461E08AE591E0F5
:1003C000E5D1CE2D6E2D669570E08AE591E05CD288
:1003D000E0FE02C061E001C060E08AE591E05CD22D
:1003E000109258018CE791E0E4D3BAE0BB2EBC0E2A
:1003F0004B2D60E08CE791E0DFD3A0923A0103C07F
:100400008CE791E0DDD3809158018823C9F389E519
:1004100091E034D1EC01F80180819181C817D907AE
:1004200009F5E1C060E070E08AE591E02DD28CE74B
:1004300091E0BFD345E061E08CE791E0BDD364E19A
:1004400070E080E090E00E94860A89E591E016D194
:10045000EC018AE591E061D361E08AE591E067D340
:100460008111DADEF801808191818C179D07D0F22D
:100470006AE070E080E090E00E94860A20C061E0BF
:1004800070E08AE591E000D28CE791E092D345E0FC
:1004900062E08CE791E090D364E170E080E090E06E
:1004A0000E94860A89E591E0E9D0EC018AE591E0B5
:1004B00034D361E08AE591E03AD38111ADDEF801F1
:1004C00080819181C817D907D0F26AE070E080E09E
:1004D00090E00E94860A20C062E070E08AE591E028
:1004E000D3D18CE791E065D341E061E08CE791E006
:1004F00063D364E170E080E090E00E94860A89E5C1
:1005000091E0BCD0EC018AE591E007D361E08AE597
:1005100091E00DD3811180DEF801808191818C17EB
:100520009D07D0F26AE070E080E090E0EFD71FC056
:1005300063E070E08AE591E0A7D18CE791E039D3E0
:1005400041E062E08CE791E037D364E170E080E065
:1005500090E0DCD789E591E091D0EC018AE591E06B
:10056000DCD261E08AE591E0E2D2811155DEF8014A
:1005700080819181C817D907D8F26AE070E080E0E5
:1005800090E0C4D78CE791E014D341E061E08CE7C0
:1005900091E012D364E170E080E090E0B7D789E5A4
:1005A00091E06CD0F80120813181C217D30719F096
:1005B000C21BD30B02C0C0E0D0E02817390799F066
:1005C000281B390BC217D30770F48CE791E0F1D2E6
:1005D00041E062E08CE791E0EFD2F6018081918109
:1005E00001969183808362E08AE591E0CFD08AE52D
:1005F00091E093D28CE791E0DCD24B2D60E08CE768
:1006000091E0DAD268EC70E080E090E07FD7FFEF15
:10061000EF1AFF0A82E0C80ED11C0E5F1F4FEBE0FD
:10062000EE16F10409F0C9CEDF91CF911F910F9121
:10063000FF90EF90DF90CF90BF90AF900895811121
:1006400006C060933A0181E0809358010895833099
:1006500009F4E2CD08957ED79EDDDEDDFECF8AE58A
:1006600091E02CC078D281E088D280E08FD261E026
:100670008AE0F6D761E08AE00C94680BCF93DF93B1
:1006800060E08AE00E94680B1EBC0DB407FEFDCF3F
:100690008EB5382F20E01EBC0DB407FEFDCF8EB501
:1006A000E901C82B61E08AE00E94680B9E01369543
:1006B00027953F70C901DF91CF910895089561E0BA
:1006C00085E0CED761E086E0CBD761E087E0C8D790
:1006D00062E08EE0C5D762E082E1C2D762E080E1ED
:1006E000BFD762E08FE0BCD762E088E0B9D762E0B4
:1006F00089E0B6C7FC01E60FF11DE60FF11D749607
:10070000808191810895FC01262F663000F13381AC
:1007100041110FC081E090E0A0E0B0E0062E04C0DF
:10072000880F991FAA1FBB1F0A94D2F7832B8383BC
:10073000089541E050E060E070E004C0440F551FB0
:10074000661F771F2A95D2F7409543231DC08381EA
:10075000442369F041E050E060E070E004C0440FE1
:10076000551F661F771F2A95D2F7482B0DC041E011
:1007700050E060E070E004C0440F551F661F771F13
:100780002A95D2F74095482343830895CF92DF926C
:10079000EF92FF920F931F93CF93DF936C01E62F9D
:1007A000F0E0E559FF4F059114918CE3E82E81E0CC
:1007B000F82EC0E0D0E01127F70161917F01A80178
:1007C0000C2E02C0559547950A94E2F741705527C3
:1007D000C60199DF2196C330D10571F7DF91CF9122
:1007E0001F910F91FF90EF90DF90CF900895EF92BF
:1007F000FF920F931F93CF93DF93DC01CFE3D1E000
:1008000080E090E06D587F4FFB01E590F49041E06F
:1008100050E060E070E09701082E02C03695279501
:100820000A94E2F720FF12C08A019B01088004C0ED
:10083000000F111F221F331F0A94D2F71296EC915A
:100840001297E02B1296EC93129712C08A019B012B
:10085000088004C0000F111F221F331F0A94D2F713
:10086000009512962C911297202312962C93129792
:10087000019621968730910571F6DF91CF911F91F6
:100880000F91FF90EF9008959C01CB016AE070E01A
:10089000BED7BC01C901ABCFFC018281662311F038
:1008A000806201C08F7D82830895CF93DF93EC0136
:1008B0009A818C81981304C09B818D81981791F047
:1008C00060E087E005D72A81209541E066E085E079
:1008D00035D72B81209541E066E085E02FD761E098
:1008E00087E0F6D68A818C838B818D83DF91CF91CF
:1008F0000895AF92BF92CF92DF92EF92FF920F9343
:100900001F93CF93DF938C01DC0153961C92EC0173
:10091000A12CB12CC12CD12C7601C3948C899D893A
:100920009B8F8A8FF501E859FF4F859194914DD6A1
:100930002C893D89FC01E21BF30B9F01F7FF03C0EB
:10094000319521953109D8015396EC915397B70110
:10095000A6010A2C04C0440F551F661F771F0A9476
:10096000D2F72C30310524F04E2B53964C9304C013
:1009700040954E23F801438B9D8B8C8BC80195DFEE
:10098000FFEFAF1ABF0A229643E0A416B10409F0A4
:10099000C5CFDF91CF911F910F91FF90EF90DF9026
:1009A000CF90BF90AF9008958F929F92AF92BF92D9
:1009B000CF92DF92EF92FF920F931F93CF93DF932B
:1009C000EC0162E08EE04CD662E082E149D662E062
:1009D00080E146D662E08FE043D662E088E040D610
:1009E00062E089E03DD68E819F81309902C08160AE
:1009F00001C08E7F9F838E838E819F81329902C03A
:100A0000826001C08D7F9F838E838E819F814999F3
:100A100002C0846001C08B7F9F838E838E819F8103
:100A2000319902C0886001C0877F9F838E838E8149
:100A30009F81189B02C0806101C08F7E9F838E833F
:100A40008E819F81199B02C0806201C08F7D9F8330
:100A50008E831F861E861D861C860E811F8140E0A8
:100A600050E020E030E080E090E0812C912C5401B7
:100A7000839475016401082E04C0CC0CDD1CEE1CAF
:100A8000FF1C0A94D2F7F601D601A095B0952A234F
:100A90003B234A235B237801082E02C0F594E79498
:100AA0000A94E2F768857985E0FE18C0DB01082E1C
:100AB00002C0B595A7950A94E2F7A0FD19C02E2BA8
:100AC0003F2B16C04E2B5F2B16C00196863091052A
:100AD00081F63D872C875F874E8712C07B01082EE9
:100AE00002C0F594E7940A94E2F7E0FCEBCF03C070
:100AF0006E2B7F2B02C06A237B2379876887E5CF23
:100B0000DF91CF911F910F91FF90EF90DF90CF90E9
:100B1000BF90AF909F908F900895CF93DF93EC019B
:100B2000E8DECE0141DFCE01DF91CF91BECEFC01E8
:100B30008681978102C0959587956A95E2F78170C5
:100B40000895FC018485958502C0959587956A95E1
:100B5000E2F78170089561E08AE0BAD561E08AE049
:100B60007FD58CB580618CBD8CB580648CBD61E017
:100B70008DE076D561E08BE073C5811103C08CB543
:100B8000806202C08CB58F7D8CBD08952CB5982FE6
:100B900093702C7F922B9CBD9DB582FB882780F99A
:100BA0009E7F982B9DBD0895CB0106C68FE991E0ED
:100BB000DBC08FE991E02AC1645C8FE991E0DAC083
:100BC000EF92FF920F931F93CF93DF931F92CDB7B6
:100BD000DEB77C010AE010E08FE991E0DCD08823E9
:100BE00009F4B6C08FE991E00BD1282F8FE991E08D
:100BF000298309D1482F2981243049F138F4223042
:100C0000D1F0F8F4213009F045C008C0263059F180
:100C100020F1273071F12830E9F531C0813029F019
:100C20008FE991E04983F5D04981D7011296ED9182
:100C3000FC91139729C0D7011496ED91FC9115975B
:100C400023C0D7011696ED91FC9117971DC0D701CF
:100C50001896ED91FC91199717C0D7011A96ED914E
:100C6000FC911B9711C0D7011C96ED91FC911D972B
:100C70000BC0D7011E96ED91FC911F9705C0D701BF
:100C80005096ED91FC915197309709F4A5CF842FA0
:100C90000995A2CF822F8A508A3030F4D70152961C
:100CA000ED91FC9153973BC0822F84518A3030F4F0
:100CB000D7015496ED91FC91559731C0822F8E51FA
:100CC0008A3030F4D7015696ED91FC91579727C0A2
:100CD000822F88528A3030F4D7015896ED91FC91DA
:100CE00059971DC0822F82538A3030F4D7015A960B
:100CF000ED91FC915B9713C0822F8C538A3030F4B6
:100D0000D7015C96ED91FC915D9709C0822F8654C6
:100D10008A3058F4D7015E96ED91FC915F97309739
:100D200009F45ACF642F099557CF243608F454CFCD
:100D3000D7019096ED91FC919197309709F44CCFA3
:100D4000822F90E084569109B80161D5099544CF6E
:100D50000F90DF91CF911F910F91FF90EF90089529
:100D6000FC01758F648F0895AB0160E070E082EA4A
:100D700091E064C1CF93C42F82EA91E0693011F40D
:100D8000ABD004C0A9D0C93009F4CAE06C2F82EA04
:100D900091E0CF91A1C0CF93DF93EC0182EA91E083
:100DA0003DD0892B39F18A8181110EC082EA91E010
:100DB00064D0888391E09A83893031F489818930C5
:100DC00019F41A82188219828A81813091F482EA98
:100DD00091E024D0892B71F082EA91E04ED0898392
:100DE0001A829881993041F4893031F4188219823D
:100DF00003C003C080E001C081E0DF91CF9108957E
:100E0000FC0180810895FC018181089549E069E039
:100E1000B1CFFC011282108211820895FC018485F9
:100E20009585FC01E05CFF4F20813181FC01EE5B88
:100E3000FF4F80819181281B390B2F733327C90104
:100E40000895FC0184859585FC01E05CFF4F40819D
:100E50005181FC01EE5BFF4F208131814217530726
:100E600041F00190F081E02DE80FF91F208130E082
:100E700002C02FEF3FEFC9010895FC0184859585DD
:100E8000FC01E05CFF4F40815181FC01EE5BFF4FB4
:100E9000208131814217530781F0A081B181A80FD1
:100EA000B91F8C91208131812F5F3F4F2F733327E2
:100EB00031832083282F30E002C02FEF3FEFC9019C
:100EC0000895FC0181A1882329F0A489B5898C911A
:100ED00086FFFBCF11A20895CF93DF93FC012685F7
:100EE0003785D901A05CBF4F8D919C9111970196D8
:100EF0008F739927E901CE5BDF4F488159818417B1
:100F00009507D9F30D90BC91A02DA20FB31F6C9340
:100F1000A685B785A05CBF4F11969C938E93A6893A
:100F2000B7892C9181E090E0078C02C0880F991F4F
:100F30000A94E2F7282B2C9381E081A30488F58999
:100F4000E02D80818064808381E090E0DF91CF910B
:100F500008951F920F920FB60F9211242F933F9373
:100F60004F938F939F93EF93FF938091C00082FDE7
:100F70001CC04091C60080914802909149020196A0
:100F80008F73992720914A0230914B028217930761
:100F900071F0E0914802F0914902E85FFD4F408313
:100FA000909349028093480202C08091C600FF914D
:100FB000EF919F918F914F913F912F910F900FBE85
:100FC0000F901F9018951F920F920FB60F92112439
:100FD0002F933F938F939F93EF93FF93209104025E
:100FE0003091050280910602909107022817390777
:100FF00031F48091C1008F7D8093C10014C0E091D5
:101000000602F0910702EC53FE4F20818091060208
:101010009091070201968F7399279093070280930E
:1010200006022093C600FF91EF919F918F913F910F
:101030002F910F900FBE0F901F901895CF92DF92B7
:10104000EF92FF92CF93DF93EC016A017B01411590
:1010500081EE580761057105F1F0EC89FD8981E0A9
:1010600090E008A002C0880F991F0A94E2F78083DD
:1010700060E079E08DE390E0A7019601DBD3215099
:1010800031094109510956954795379527952115FD
:1010900080E1380790F0EC89FD89108260E874E8FF
:1010A0008EE190E0A7019601C5D321503109410995
:1010B00051095695479537952795E889F9893083E1
:1010C000EA89FB89208319A2EE89FF89408181E0AA
:1010D00090E09C010C8C02C0220F331F0A94E2F7AF
:1010E000422B4083EE89FF8940819C010D8C02C018
:1010F000220F331F0A94E2F7422B4083EE89FF89C7
:1011000040819C010E8C02C0220F331F0A94E2F72B
:10111000422B4083EE89FF8920810F8C02C0880F0B
:10112000991F0A94E2F7809582238083DF91CF9103
:10113000FF90EF90DF90CF9008951092A50110924C
:10114000A40188EE93E0A0E0B0E08093A601909324
:10115000A701A093A801B093A9018BE491E090931B
:10116000A3018093A20188E092E09093AF01809365
:10117000AE0184EC91E09093B1018093B00185ECD5
:1011800090E09093B3018093B20184EC90E090934F
:10119000B5018093B40180EC90E09093B701809307
:1011A000B60181EC90E09093B9018093B80182EC94
:1011B00090E09093BB018093BA0186EC90E090930D
:1011C000BD018093BC0184E08093BE0183E08093E5
:1011D000BF0187E08093C00185E08093C10181E079
:1011E0008093C2010895CF92DF92EF92FF920F9306
:1011F0001F93CF93DF936C01EB017A01E60EF71E8C
:1012000000E010E00BC06991D601ED91FC910190D6
:10121000F081E02DC6010995080F191FCE15DF05D5
:1012200091F7C801DF91CF911F910F91FF90EF903F
:10123000DF90CF9008956115710581F0DB010D906D
:101240000020E9F7AD0141505109461B570BDC0165
:10125000ED91FC910280F381E02D099480E090E013
:101260000895DC01ED91FC910190F081E02D09944D
:101270000F931F93CF93DF93EC016DE0F2DF8C01AE
:101280006AE0CE01EEDF9C01200F311FC901DF9122
:10129000CF911F910F9108954F925F926F927F921D
:1012A0009F92AF92BF92CF92DF92EF92FF920F93F5
:1012B0001F93CF93DF93CDB7DEB7A1970FB6F89406
:1012C000DEBF0FBECDBF5C016A017B01922E19A269
:1012D00081E0821710F08AE0982E8E010F5D1F4F7B
:1012E000492C512C612C712CC701B601A30192012C
:1012F000A1D28C2D929E80191124015011098A309F
:1013000014F4805D01C0895CF801808369017A0171
:10131000C114D104E104F10439F7B801C5018BDF30
:10132000A1960FB6F894DEBF0FBECDBFDF91CF916F
:101330001F910F91FF90EF90DF90CF90BF90AF90F3
:101340009F907F906F905F904F9008952115310589
:1013500041F4DC01ED91FC910190F081E02D642FCE
:1013600009949ACF0F931F93CF93DF93EC019A01C7
:10137000AB0160E070E0EADF8C01CE0179DF98011B
:10138000280F391FC901DF91CF911F910F91089547
:101390004F925F926F927F92AF92BF92CF92DF9205
:1013A000EF92FF920F931F93CF93DF93CDB7DEB7EA
:1013B00029013A01621B730B840B950B29893A8929
:1013C0004B895C892A193B094C095D09298B3A8BA9
:1013D0004B8B5C8B9B01AC0169897A898B899C89D9
:1013E000F3D1E418F50806091709A801970144D2BA
:1013F0002A0D3B1D4C1D5D1DB901CA01DF91CF9126
:101400001F910F91FF90EF90DF90CF90BF90AF9022
:101410007F906F905F904F900895382F20E0262B9B
:10142000C90108951F920F920FB60F9211242F93A6
:101430003F938F939F93AF93BF9380914C02909172
:101440004D02A0914E02B0914F0230915402232FD1
:101450002D5F2D3720F40196A11DB11D05C0232F4E
:101460002A570296A11DB11D2093540280934C026D
:1014700090934D02A0934E02B0934F028091500280
:1014800090915102A0915202B09153020196A11D78
:10149000B11D8093500290935102A0935202B093D9
:1014A0005302BF91AF919F918F913F912F910F90D8
:1014B0000FBE0F901F9018950F931F939FB7F8942E
:1014C000009150021091510220915202309153022A
:1014D00086B5A89B06C08F3F21F00F5F1F4F2F4F8F
:1014E0003F4F9FBF322F212F102F0027080F111DB4
:1014F000211D311D42E0000F111F221F331F4A958D
:10150000D1F7B801C9011F910F910895CF92DF92D1
:10151000EF92FF92CF93DF936B017C01CDDFEB0164
:101520000DC0CADF6C1B7D0B683E734038F081E054
:10153000C81AD108E108F108C851DC4FC114D10420
:10154000E104F10471F7DF91CF91FF90EF90DF900C
:10155000CF900895789484B5826084BD84B581600D
:1015600084BD85B5826085BD85B5816085BDEEE6AB
:10157000F0E0808181608083E1E8F0E0108280818A
:1015800082608083808181608083E0E8F0E08081F8
:1015900081608083E1EBF0E0808184608083E0EB18
:1015A000F0E0808181608083EAE7F0E08081846000
:1015B000808380818260808380818160808380815C
:1015C000806880831092C10008958E3008F08E509C
:1015D000877020913B0140E4249F90011124822BCD
:1015E00080937C0080917A00806480937A0080915F
:1015F0007A0086FDFCCF2091780030917900932FFE
:1016000080E0AC01422B9A01C9010895833069F052
:1016100028F48130A1F0823011F514C08630B1F089
:101620008730C1F08430D9F404C0809180008F7776
:1016300003C0809180008F7D80938000089584B5E1
:101640008F7702C084B58F7D84BD08958091B000EE
:101650008F7703C08091B0008F7D8093B000089594
:10166000CF93DF9390E0FC01E454FF4F4491FC01E1
:10167000E053FF4F8491882341F190E0880F991F38
:10168000FC01E251FF4F25913491D9018C519F4FBC
:10169000FC0185919491C82FD92F9FB7F8948C9114
:1016A000611106C0409584238C938881842308C0EF
:1016B000623041F4242F209582238C938881842BDF
:1016C000888302C0842B8C939FBFDF91CF910895B4
:1016D0000F931F93CF93DF931F92CDB7DEB7282FC1
:1016E00030E0F901E855FF4F8491F901E454FF4FD0
:1016F0001491F901E053FF4F04910023C9F08823AE
:1017000019F0698383DF6981E02FF0E0EE0FFF1F9E
:10171000EC51FF4F85919491DC019FB7F8948C9127
:10172000611103C01095812301C0812B8C939FBF51
:101730000F90DF91CF911F910F910895BF92CF929B
:10174000DF92EF92FF920F931F93CF93DF93C82EF8
:10175000D62EB42EC7E0D0E0022F10E087E0E82EAE
:10176000F12CB1100AC0F701EC1BFD0BB80102C04F
:1017700075956795EA95E2F707C0B8010C2E02C08F
:10178000759567950A94E2F7617077278C2DA0DF35
:1017900061E08D2D9DDF60E08D2D9ADF219708F7A8
:1017A000DF91CF911F910F91FF90EF90DF90CF903D
:1017B000BF900895F89497C0F999FECF92BD81BD6E
:1017C000F89A992780B50895DB018F939F936FD086
:1017D000BF91AF91A29F800D911DA39F900DB29FCD
:1017E000900D11240895AA1BBB1B51E107C0AA1F2D
:1017F000BB1FA617B70710F0A61BB70B881F991FB2
:101800005A95A9F780959095BC01CD01089597FB55
:10181000072E16F4009406D077FD08D0E4DF07FC0D
:1018200005D03EF4909581959F4F089570956195F0
:101830007F4F0895A1E21A2EAA1BBB1BFD010DC00C
:10184000AA1FBB1FEE1FFF1FA217B307E407F50770
:1018500020F0A21BB30BE40BF50B661F771F881F4C
:10186000991F1A9469F760957095809590959B01E2
:10187000AC01BD01CF010895052E97FB16F400942D
:1018800006D057FD0CD0D6DF07FC09D07EF490952A
:101890008095709561957F4F8F4F9F4F089550951C
:1018A0004095309521953F4F4F4F5F4F08950FD092
:1018B000A59F900DB49F900DA49F800D911D1124A4
:1018C0000895EE0FFF1F0590F491E02D0994A29F5B
:1018D000B001B39FC001A39F01D0B29F700D811DC5
:0A18E0001124911D0895F894FFCF24
:1018EA000100000000009A013303CD0466060008D7
:1018FA009A09330BCD0C660EFF0FFF0F02085C0826
:10190A00B30809096309BC09130A6C0AC90A1C0B42
:10191A00730B0000000000000000FF010504030033
:10192A0001020304070605000000006C07F3080E15
:08193A00073D072107610700CA
:00000001FF
